:1000000002003E080808090909E7F426F460012205
:100010001819E7F426F46001221819E7F426F460B1
:1000200001221819E7F426F4600122C3B322E63353
:10003000F608E633F608E633F608E633F6220075EE
:10004000891153880F758A00758C00758B00758D2A
:10005000007A4020B4FD30B4FDD28C20B4FDC28CB7
:10006000D28E30B4FDC28EDAF0E58A24BDF530E5DB
:100070008C3400F531E58B2440F534E58D3400F502
:10008000357538A6753905753CA9753D0200E53012
:100090008538F0A4F54485F045754600754700E5C0
:1000A000318538F0A4754800F54985F04A754B0054
:1000B00000C3E5443548F544E5453549F545E54691
:1000C000354AF546E547354BF54700E5308539F0CB
:1000D000A4754800F54985F04A754B0000C3E54416
:1000E0003548F544E5453549F545E546354AF54693
:1000F000E547354BF54700E5318539F0A4754800F3
:10010000754900F54A85F04B00C3E5443548F54490
:10011000E5453549F545E546354AF546E547354B6C
:10012000F547000000E534853CF0A4F54C85F04D22
:10013000754E00754F00E535853CF0A4755000F50F
:100140005185F05275530000C3E54C3550F54CE530
:100150004D3551F54DE54E3552F54EE54F3553F5DC
:100160004F00E534853DF0A4755000F55185F052FF
:1001700075530000C3E54C3550F54CE54D3551F550
:100180004DE54E3552F54EE54F3553F54F00E5350B
:10019000853DF0A4755000755100F55285F053006F
:1001A000C3E54C3550F54CE54D3551F54DE54E3533
:1001B00052F54EE54F3553F54F000000C3E530359D
:1001C00034F530E5313535F531E5323536F532E5A2
:1001D000333537F533007844794C1103403000C390
:1001E000E54C9544F54CE54D9545F54DE54E954668
:1001F000F54EE54F9547F54F00E54CF544E54DF5D7
:1002000045E54EF546E54FF5477FFF02022B00C35B
:10021000E544954CF544E545954DF545E546954E47
:10022000F546E547954FF547007F00007A20784472
:10023000112E7858112E7858793000110300502271
:100240007854112E00C3E5589530F558E55995318D
:10025000F559E55A9532F55AE55B9533F55B0002A1
:1002600002667854112EDAC600C3E5783554F57865
:10027000E5793555F579E57A3556F57AE57B3557E3
:10028000F57B000EEE600302034E007A20E55C254C
:100290005CD4F55CE55D355DD4F55DE55E355ED439
:1002A000F55EE55F355FD4F55F7879112E501CE57A
:1002B0005C2401D4F55CE55D3400D4F55DE55E3485
:1002C00000D4F55EE55F3400D4F55FDAC0757800E0
:1002D000757900757A00757B00757C00E55CF5909A
:1002E00053890F438920758DFD53877F759840D2C0
:1002F0008EC298C299EF6005742D0202FF7420F53A
:10030000993099FDC299E55D54F0C42430F59930D7
:1003100099FDC299E55D540F2430F5993099FDC2DD
:1003200099E55C54F0C42430F5993099FDC2997474
:100330002EF5993099FDC299E55C540F2430F5995A
:100340003099FDC299740DF5993099FDC2997830B4
:0B0350007A3C760008DAFB010080FE1A
:00000001FF
